:040000000200833245
:01000B0032C2
:0100130032BA
:01001B0032B2
:0100230032AA
:20002B00322B2B2B20464C2053747564696F204D4944492052656D6F746520436F6E7472C3
:20004B006F6C6C65722056312E3031202F20415438394332303531202F20284329205374D7
:20006B006566616E204861726173696D2030332F32303038202B2B2B758124758920758D9F
:20008B00FF75884075987CD29975A800C2997590FF75B0FF75080F74902508F50974B02581
:2000AB0008F50A7520007521007522007523001200C812019512026212032F80F2C2B3E5CC
:2000CB0090F47003D2B32285090830E018750C30750D7F120411120429750D0012041130C8
:2000EB0090FD12042930E118750C32750D7F120411120429750D001204113091FD12042940
:20010B0030E218750C34750D7F120411120429750D001204113092FD12042930E318750C3B
:20012B0035750D7F120411120429750D001204113093FD12042930E418750C37750D7F1279
:20014B000411120429750D001204113094FD12042930E518750C39750D7F12041112042949
:20016B00750D001204113095FD12042930E618750C3B750D7F120411120429750D001204E1
:20018B00113096FD120429D2B322C2B5E590F47003D2B52285090830E018750C3C750D7F22
:2001AB00120411120429750D001204113090FD12042930E118750C3E750D7F120411120403
:2001CB0029750D001204113091FD12042930E218750C40750D7F120411120429750D00125F
:2001EB0004113092FD12042930E318750C41750D7F120411120429750D001204113093FD24
:20020B0012042930E418750C43750D7F120411120429750D001204113094FD12042930E57F
:20022B0018750C45750D7F120411120429750D001204113095FD12042930E618750C477559
:20024B000D7F120411120429750D001204113096FD120429D2B522C2B4E590F47003D2B475
:20026B002285090830E018750C36750D7F120411120429750D001204113090FD12042930A0
:20028B00E118750C31750D7F120411120429750D001204113091FD12042930E218750C33BD
:2002AB00750D7F120411120429750D001204113092FD12042930E318750C38750D7F12042A
:2002CB0011120429750D001204113093FD12042930E418750C46750D7F120411120429754C
:2002EB000D001204113094FD12042930E518750C44750D7F1204111204293095FD750D0022
:20030B0012041112042930E618750C42750D7F120411120429750D001204113096FD120492
:20032B0029D2B422C2B7E590F47003D2B72230E01B850908750C3D750D7F120411120429FB
:20034B00750D001204113090FD12042930E11B850A08750C13750D7F120411120432309165
:20036B00FD750D0012041112042930E21B850A08750C14750D7F1204111204323092FD7590
:20038B000D0012041112042930E31B850908750C3F750D7F120411120429750D001204114B
:2003AB003093FD12042930E41B850A08750C16750D7F120411120429750D00120411309402
:2003CB00FD12042930E51E850A08750C15750D7F120411120432750D0012041112042930EE
:2003EB0095FD12042930E61B850A08750C17750D7F120411120429750D001204113096FDEE
:20040B00120429D2B7228508993099FDC299850C993099FDC299850D993099FDC2997AC3CC
:10042B007989D9FEDAFC227A0279EED9FEDAFC223E
:00043B01C0
